:1000000028C042C022C240C0E1C13EC03DC03CC089
:100010003BC03AC039C05CC337C036C035C034C0FD
:1000200033C00000000000040302010000000102D0
:1000300004081020408004020108010101010101AF
:1000400001010202020200003B00380000003A00F9
:10005000370011241FBECFE5D2E0DEBFCDBF10E0D8
:10006000A0E6B0E0E6EDFBE002C005900D92A437FB
:10007000B107D9F720E0A4E7B0E001C01D92AC3988
:10008000B207E1F7A9D4A5C5BBCFEF92FF920F93BA
:100090001F93CF93DF930DE610E0C0E0D0E0EE2495
:1000A000E394F12CC7010C2E01C0880F0A94EAF7E3
:1000B00060917B006823F80181918F0119D421960A
:1000C000C830D10579F7DF91CF911F910F91FF9043
:1000D000EF900895DF92EF92FF920F931F93CF93CB
:1000E000DF93C0E0D0E0082F10E08AE2D82E9CE138
:1000F000E92E29E4F22EC017D107D4F4D0927B0068
:10010000C4DF64E670E080E090E053D3E0927B00CF
:10011000BCDF64E670E080E090E04BD3F0927B00BF
:10012000B4DF64E670E080E090E043D32196E3CF53
:10013000DF91CF911F910F91FF90EF90DF90089585
:100140000F931F93CF93DF93062F10E0C82FD0E0BB
:10015000CB59DF4F101799F010927B0096DF6AEFB2
:1001600070E080E090E025D3888180937B008DDF74
:100170006AEF70E080E090E01CD31F5FEBCFDF916F
:10018000CF911F910F910895CF93DF93CAE0DBE6E3
:1001900010927B007ADF64E670E080E090E009D3A3
:1001A000D0937B0072DF64E670E080E090E001D3E2
:1001B000C15071F7DF91CF9108951092770010929E
:1001C00078001092790010927A0080E28093760095
:1001D000F89414BE81B5886181BD80E481BD7894B6
:1001E000809176001816E4F3F89414BE81B580610E
:1001F00081BD11BC78940895CF93DF93D82FC62F7B
:1002000069E18CE790E032D16D2F8CE790E034D13A
:100210006C2F8CE790E030D18CE790E0DF91CF91AC
:1002200052C1CF93DF93D82FC62F69E18CE790E0BE
:100230001DD16D2F8CE790E01FD18CE790E043D16A
:100240004C2F69E18CE790E040D18CE790E053D1EE
:1002500097FD80E0DF91CF91089561E081E3E1DFD8
:1002600080917400813009F435DF26E030E040E011
:1002700050E060E070E0CB018ED3862F6093750074
:1002800090917400913069F4E62FF0E0EB59FF4F44
:10029000808180937B00F9DE68E873E180E090E084
:1002A00006C063E04DDF60ED77E080E090E081D252
:1002B00010927B00EADE85B7877E806185BF85B7B7
:1002C000806285BF85B7806285BF889585B78F7D41
:1002D00085BF6AE070E080E090E06BD285B78F7DEB
:1002E00085BF08956FE380E287DF60E083E284DF0B
:1002F00060E08FE181DF6FE380E37EDF62E082E335
:100300007BDF61E083E378DF65E188E375DF67E049
:1003100089E372DF68E08AE36FDF68E08BE36CDF1C
:1003200068E08CE369DF60E18DE366DF61E084E231
:1003300078DF837F682F686084E25EDF60E882E2B6
:100340005BDF60E085E258CFCF93DF93CDE6D0E06E
:1003500061E089918FD280E0C537D807C9F760E0A6
:1003600080E888D280E888B916B881E082BB1ABEDE
:1003700080E18BBF78948CE790E077D06AE070E002
:1003800080E090E016D261E08FE04BDF833309F02C
:10039000FBDEA8DF64E670E080E090E00AD261E076
:1003A0008DE23FDF87FF04C081E08093740002C0CC
:1003B0001092740002DF8091770090917800A091F4
:1003C0007900B0917A00DF91CF91C6C21F920F924F
:1003D0000FB60F9211242F938F939F93AF93BF93D8
:1003E0008091760081508093760080917700909183
:1003F0007800A0917900B0917A00BA2FA92F982F98
:1004000088278093770090937800A0937900B09329
:100410007A002CB58091770090917800A0917900B6
:10042000B0917A0082278093770090937800A09310
:100430007900B0937A00BF91AF919F918F912F91E6
:100440000F900FBE0F901F9018951F920F920FB62E
:100450000F9211248F9381E0809364001ABE8F91D4
:100460000F900FBE0F901F90189550C010927F00F4
:10047000660F609380000895E0917F00E13150F4B1
:10048000EF5FE0937F00F0E0E058FF4F608381E092
:1004900090E0089580E090E00895CF93C62F60919A
:1004A0007F006F5F80E890E0E5D010927F008823A6
:1004B00029F0CC2329F0E1D0811102C0CF9131C0C5
:1004C00080E0CF91089561E0E8CF10927E004093E4
:1004D0007D00660F862F81608093800061E0640F4D
:1004E00080E890E0C7D0882319F0C7D0811101C0FF
:1004F00018C080E00895E0917E00EF5FE0937E00F9
:10050000F0E0E058FF4F808190E00895DE9ADC9A99
:10051000D49AD69A8FEF8FB98AE28DB980EF8EB9CF
:1005200008958091920008958EB98BE29DE09A958E
:10053000F1F700008DB9CC9BFECF9AE09A95F1F7C8
:1005400000C08DB9769BF2CF8DE08A95F1F700005F
:100550008FB19FEF9FB9D69A0895DC9ADC9BFECFAE
:100560008DE08A95F1F70000DE988AE08A95F1F730
:1005700000C0DC98DE9A779905C083E080939200F2
:1005800080E0089581E00895AF92BF92CF92DF920C
:10059000EF92FF920F931F93CF93DF938C01E62E80
:1005A00080919200816080939200F801908190FD8B
:1005B00003C0826080939200D0DF882309F44FC08B
:1005C000FE2CE801BB24BA94AA24A3948091920043
:1005D00083709E012F5F3F4F6901882361F1DC9892
:1005E00088818FB980EFA0DFD6988EEF9DDF909144
:1005F000920080FF0BC0892F817090FF05C081E0C1
:100600008093920080E02BC092E00EC0892F85700D
:10061000843069F4F801808181608083A092920027
:100620009CDF811116C09AE09093920018C09E7FC3
:10063000909392000CC0D69880EF76DF8883F1E02B
:10064000FF1202C0BFB801C01FB88EEF6DDFE60118
:1006500002C0FE2CE801FA94F110B8CF81E0DF91DE
:10066000CF911F910F91FF90EF90DF90CF90BF90AF
:10067000AF9008951092920087CFDE98DC9ACC9BC1
:10068000FECF8AE08A95F1F700C0DE9A8DE08A9568
:10069000F1F700009EB1892F807295FD04C094E0AF
:1006A00090939200089581E008958EB5887F8EBD65
:1006B0008FB581608FBD8FB58D7F8FBD8EB5877FE4
:1006C0008EBD8EB58F7E8EBD8EB583608EBD089536
:1006D0001F920F920FB60F9211242F933F938F9377
:1006E0009F93AF93BF938091940090919500A091B8
:1006F0009600B09197003091930026E0230F2D379C
:1007000030F029E8230F0396A11DB11D03C0029606
:10071000A11DB11D209393008093940090939500A8
:10072000A0939600B09397008091980090919900C3
:10073000A0919A00B0919B000196A11DB11D8093DC
:10074000980090939900A0939A00B0939B00BF915A
:10075000AF919F918F913F912F910F900FBE0F906E
:100760001F9018953FB7F894809198009091990048
:10077000A0919A00B0919B0022B708B600FE05C078
:100780002F3F19F00196A11DB11D3FBFBA2FA92F10
:10079000982F8827820F911DA11DB11DBC01CD018D
:1007A00043E0660F771F881F991F4A95D1F7089578
:1007B0000895CF92DF92EF92FF92CF93DF936B0178
:1007C0007C01D0DFEB01C114D104E104F104A1F0FC
:1007D000EFDFC8DF6C1B7D0B683E7340A0F3C114D4
:1007E000D104E104F10479F381E0C81AD108E108E9
:1007F000F108C851DC4FEDCFDF91CF91FF90EF9022
:10080000DF90CF90089580B7826080BF80B781600D
:1008100080BF83B7887F836083BF789489B7816006
:1008200089BF43DF86B18877866886B9379A08958D
:10083000813031F480B78F7780BF80B78F7B07C05E
:10084000823039F480B78F7D80BF80B78F7E80BFC4
:100850000895833031F48FB58F778FBD8FB58F7B3F
:1008600007C0843031F48FB58F7D8FBD8FB58F7EFB
:100870008FBD0895CF93DF9387FD8F7790E0FC01C4
:10088000E25DFF4F2491FC01E65CFF4F84918823D9
:1008900061F190E0880F991FFC01E45BFF4FC59167
:1008A000D491FC01EA5BFF4FA591B491611109C09D
:1008B0009FB7F8948881209582238883EC912E231A
:1008C0000BC0623061F49FB7F8948881322F309565
:1008D00083238883EC912E2B2C939FBF06C08FB768
:1008E000F894E8812E2B28838FBFDF91CF91089554
:1008F0001F93CF93DF93162F87FD8F77282F30E03C
:10090000F901EE5DFF4F8491F901E25DFF4FD49153
:10091000F901E65CFF4FC491CC23D1F0811188DF4F
:10092000EC2FF0E0EE0FFF1FEA5BFF4FA591B491B3
:10093000111108C09FB7F8948C91D095D823DC93FF
:100940009FBF06C08FB7F894EC91DE2BDC938FBF6E
:10095000DF91CF911F910895009721F0BC0180E0B5
:1009600090E02EC10895CF92DF92EF92FF92611531
:1009700071058105910539F06B017C01D4D0A70187
:10098000960149D003C060E070E0CB01FF90EF908A
:10099000DF90CF900895CF92DF92EF92FF920F9366
:1009A0001F9362177307840795077CF489019A01E6
:1009B0006B017C01C901B8016C197D098E099F0981
:1009C000D2DF6C0D7D1D8E1D9F1D1F910F91FF901D
:1009D000EF90DF90CF90089581B781BF14DFB4DC32
:1009E0003CDCFECFEE27FF27AA27BB2708C0A20FBB
:1009F000B31FE41FF51F220F331F441F551F969589
:100A000087957795679598F37040A9F7009799F7C0
:100A1000BD01CF010895052E97FB16F400940FD069
:100A200057FD05D014D007FC02D046F408C05095FD
:100A30004095309521953F4F4F4F5F4F08959095CA
:100A40008095709561957F4F8F4F9F4F0895A1E2DC
:100A50001A2EAA1BBB1BFD010DC0AA1FBB1FEE1F38
:100A6000FF1FA217B307E407F50720F0A21BB30B83
:100A7000E40BF50B661F771F881F991F1A9469F7FF
:100A800060957095809590959B01AC01BD01CF015B
:100A900008958F929F92AF92BF92CF92DF92EF9282
:100AA000FF92CF93DF93EC01688179818A819B81EA
:100AB000611571058105910521F464E279ED8BE5FD
:100AC00097E02DE133EF41E050E0A5DF49015A0105
:100AD00027EA31E440E050E085DF6B017C012CEE39
:100AE00034EF4FEF5FEFC501B4017CDFDC01CB01D8
:100AF0008C0D9D1DAE1DBF1DB7FF03C00197A10941
:100B0000B04888839983AA83BB83BC01CD019F77BA
:100B1000DF91CF91FF90EF90DF90CF90BF90AF909B
:100B20009F908F9008958F929F92AF92BF92CF9295
:100B3000DF92EF92FF92609160007091610080916E
:100B4000620090916300611571058105910521F4A2
:100B500064E279ED8BE597E02DE133EF41E050E081
:100B60005ADF49015A0127EA31E440E050E03ADF18
:100B70006B017C012CEE34EF4FEF5FEFC501B40148
:100B800031DFDC01CB018C0D9D1DAE1DBF1DB7FFFC
:100B900003C00197A109B048809360009093610061
:100BA000A0936200B0936300BC01CD019F77FF90DA
:100BB000EF90DF90CF90BF90AF909F908F9008956F
:100BC0006093600070936100809362009093630073
:060BD0000895F894FFCF28
:100BD600010000000108222A636B771C490A0908F4
:040BE60007010203FE
:00000001FF
